:020000040000FA
:1000000055D000000000000048D0000000000000B3
:100010000000000000000000D8CFDFF0E8CFDEF0E5
:10002000E0CFDDF0EACFDAF0E9CFD9F09EAA02D036
:100030009DBA4FD39EA802D09DB83AD3FF00D9C035
:10004000E9FFDAC0EAFFDDC0E0FFDEC0E8FFDFC0A5
:04005000D8FF1000C5
:020054000000AA
:06009A00EACFDCF0E9CF23
:0C00A000DBF0F2A402D0F2BA14D0FF0092
:0400AC00926A936A57
:1000B000946A0C0E006E98EC02F027EC04F064ECED
:1000C00000F029EC04F0FDD7C00ED56EF184F28A61
:1000D0001200F294A00ED66E010E815F000E805BBE
:1000E00080BFA9EC00F0010E8B5F000E8A5B8ABF17
:1000F000B7EC00F0010E955F000E945B94BFC5EC69
:1001000000F0010E9F5F000E9E5B9EBFD3EC00F0DF
:10011000010EA95F000EA85BA8BFE1EC00F0010E84
:10012000B35F000EB25BB2BFEFEC00F0010EBD5F3B
:10013000000EBC5BBCBFFDEC00F0010EC75F000E03
:10014000C65BC6BF0BEC01F0DBC0E9FFDCC0EAFF19
:1001500011008ABE06D08A8E8251806F8351816FD2
:1001600012008A9E8451806F8551816F12008ABC73
:1001700006D08A8C8C518A6F8D518B6F12008A9CAD
:100180008E518A6F8F518B6F12008ABA06D08A8A7D
:100190009651946F9751956F12008A9A9851946F67
:1001A0009951956F12008AB806D08A88A0519E6F27
:1001B000A1519F6F12008A98A2519E6FA3519F6F09
:1001C00012008AB606D08A86AA51A86FAB51A96FD1
:1001D00012008A96AC51A86FAD51A96F12008AB473
:1001E00006D08A84B451B26FB551B36F12008A94AD
:1001F000B651B26FB751B36F12008AB206D08A827D
:10020000BE51BC6FBF51BD6F12008A92C051BC6F0E
:10021000C151BD6F12008AB006D08A80C851C66F26
:10022000C951C76F12008A90CA51C66FCB51C76FB0
:10023000120086C0D0F087C0D1F088C0D5F089C048
:10024000D6F03AEC03F0D0C082F0D1C083F08351F5
:10025000875D856F82518659846F120090C0D0F0FF
:1002600091C0D1F092C0D5F093C0D6F03AEC03F033
:10027000D0C08CF0D1C08DF08D51915D8F6F8C51BD
:1002800090598E6F12009AC0D0F09BC0D1F09CC0E4
:10029000D5F09DC0D6F03AEC03F0D0C096F0D1C0B6
:1002A00097F097519B5D996F96519A59986F1200EC
:1002B000A4C0D0F0A5C0D1F0A6C0D5F0A7C0D6F09C
:1002C0003AEC03F0D0C0A0F0D1C0A1F0A151A55DDF
:1002D000A36FA051A459A26F1200AEC0D0F0AFC05E
:1002E000D1F0B0C0D5F0B1C0D6F03AEC03F0D0C038
:1002F000AAF0D1C0ABF0AB51AF5DAD6FAA51AE5912
:10030000AC6F1200B8C0D0F0B9C0D1F0BAC0D5F00F
:10031000BBC0D6F03AEC03F0D0C0B4F0D1C0B5F019
:10032000B551B95DB76FB451B859B66F1200C2C0BC
:10033000D0F0C3C0D1F0C4C0D5F0C5C0D6F03AECFF
:1003400003F0D0C0BEF0D1C0BFF0BF51C35DC16FDC
:10035000BE51C259C06F1200CCC0D0F0CDC0D1F098
:10036000CEC0D5F0CFC0D6F03AEC03F0D0C0C8F084
:10037000D1C0C9F0C951CD5DCB6FC851CC59CA6F3E
:100380001200022A024E0FD0024E18D0024E21D087
:10039000024E2AD0024E33D0024E3CD0024E45D0FF
:1003A000024E4ED01200034405E08980886F896BAD
:1003B00040D71200899088693CD71200034405E0B9
:1003C0008982926F936B4AD712008992926946D7BD
:1003D0001200034405E089849C6F9D6B54D7120082
:1003E00089949C6950D71200034405E08986A66F62
:1003F000A76B5ED712008996A6695AD712000344EC
:1004000005E08988B06FB16B68D712008998B06930
:1004100064D71200034405E0898ABA6FBB6B72D7B8
:100420001200899ABA696ED71200034405E08B8ADC
:10043000C46FC56B7CD712008B9AC46978D7120041
:10044000034405E08B88CE6FCF6B86D712008B9864
:10045000CE6982D71200022A024E0FD0024E16D069
:10046000024E1DD0024E24D0024E2BD0024E32D06E
:10047000024E39D0024E40D01200889103BC8881D0
:10048000039C0344E846896FD4D61200929103BCC2
:100490009281039C0344E846936FE0D612009C913E
:1004A00003BC9C81039C0344E8469D6FECD612007C
:1004B000A69103BCA681039C0344E846A76FF8D627
:1004C0001200B09103BCB081039C0344E846B16FB5
:1004D00004D71200BA9103BCBA81039C0344E846D6
:1004E000BB6F10D71200C49103BCC481039C0344AA
:1004F000E846C56F1CD71200CE9103BCCE81039C89
:100500000344E846CF6F28D71200036602D08B96CB
:1005100012008B861200036602D08B9212008B822F
:100520001200036602D08B9412008B84120012001A
:10053000826B8C6B966BA06BAA6BB46BBE6BC86B3B
:10054000836B8D6B976BA16BAB6BB56BBF6BC96B23
:1005500085698F699969A369AD69B769C169CB6913
:100560007F0E846F8E6F986FA26FAC6FB66FC06F87
:10057000CA6F806B8A6B946B9E6BA86BB26BBC6B03
:10058000C66BE86A816FE82AE82A8B6FE82AE82AB6
:10059000956FE82AE82A9F6FE82AE82AA96FE82AD7
:1005A000E82AB36FE82AE82ABD6FE82AE82AC76F6D
:1005B0008A9E8A9C8A9A8A988A968A948A928A9033
:1005C000886B926B9C6BA66BB06BBA6BC46BCE6B7B
:1005D000896B936B9D6BA76BB16BBB6BC56BCF6B63
:1005E000020E866F906F9A6FA46FAE6FB86FC26F76
:1005F000CC6F000E876F916F9B6FA56FAF6FB96F58
:10060000C36FCD6F882B922B9C2BA62B922B9C2BF0
:10061000A62B9C2BA62BA62B19EC01F02EEC01F09F
:1006200043EC01F058EC01F06DEC01F082EC01F0CC
:1006300097EC01F0ACEC01F089908992899489964D
:100640008998899A8B9A8B9812000350100DF45058
:10065000866F906F9A6FA46FAE6FB86FC26FCC6FDA
:10066000F350876F916F9B6FA56FAF6FB96FC36FBB
:10067000CD6F1200D1C0D4F0D151D603F4CFD2F057
:10068000F3CFD3F0D051D503F4CFD0F0F3CFD1F0E6
:10069000D603F350D227F450D123E86AD023D451A3
:1006A000D503F350D227F450D123E86AD023000CAD
:1006B0000BA202D09D9802D089D8AD6ED9C0E9FFB7
:1006C000DAC0EAFFDDC0E0FFDEC0E8FFDFC0D8FF30
:1006D0001000ABB207D0ABB40BD00BB410D0AE50FF
:1006E00058D8ECD7AB98AB880468FA0E32D8E6D766
:1006F000AE50AB98AB880468FB0E2BD8DFD7AE505A
:100700000468FB0E26D8DAD7800E94124F0EAF6E17
:10071000240EAC6E900EAB6E0B6A09D811D89D8872
:100720009D8A9F989F9AD08EF28EF28C1200000EB6
:100730000F6E116E170E106E126E0B900B82120060
:10074000000E136E156E270E146E166E0B940B862C
:1007500012009D980BB01BD011C0EAFF12C0E9FF38
:10076000EE6E000EEA6205D0270EE96202D000EEBE
:1007700017F0EACF11F0E9CF12F00F50116204D058
:100780001050126201D00B800B929D8812009D8840
:1007900012000BB41AD015C0EAFF16C0E9FFEE6EC6
:1007A000000EEA6205D0370EE96202D000EE27F0B3
:1007B000EACF15F0E9CF16F01350156204D01450AB
:1007C000166201D00B840B96120012000BB21CD0E3
:1007D0000FC0EAFF10C0E9FFEECF0EF0000EEA6294
:1007E00005D0270EE96202D000EE17F0EACF0FF035
:1007F000E9CF10F011500F6204D01250106201D0F6
:100800000B820B900E501200000C9D9A0BB61DD05F
:1008100013C0EAFF14C0E9FFEECF0DF0000EEA624C
:1008200005D0370EE96202D000EE27F0EACF13F0D0
:10083000E9CF14F01550136204D01650146201D0A1
:100840000B860B940D509D8A12009D8A000C84EF3C
:1008500003F00BB61200D9DF056E05AE0CD0016EA9
:1008600001AC05D0010E01AA076E066A1200020E45
:10087000076E066A1200066610D005C002F0062A4E
:100880000650075C01E0120000500118096ED00EFE
:10089000095C01E197EF02F0120005C003F0066A5F
:1008A00000500118096E900E095C01E19BEF04F005
:1008B000800E095C01E19AEF04F0B00E095C01E1E1
:1008C00063EF04F012007B0E025C01E198EF02F08E
:0E08D0007F0E025C01E1FF00AEEF04F01200AB
:0208DE00C00E4A
:1008E000E83EFED71200D76BD7C0D8F0D82B8B804C
:1008F0006FEC04F0D82FFCD78B90D7C0D8F06FECFA
:1009000004F0D83FFCD78B90D73FEED7FF0ED70E21
:10091000D7C0D8F0D82B8B806FEC04F0D82FFCD741
:100920008B90D7C0D8F06FEC04F0D83FFCD7D72F0E
:04093000EFD71200EB
:0C093400036A0250470807E602503F0823
:1009400004E7E86CE806026E1CD5590E025CE84E1E
:10095000DCD5E84EE0D5E84EE4D512000250470859
:1009600007E602503F0804E7E86CE806026E73D51C
:0C0970000250160802E125EF03F012000F
:020000040030CA
:0E000000FFFEFDFEFFFFFAFFFFFFFFFFFFFF09
:00000001FF
